:01000000FF00
:05F1FB00FFFFFFFFFF14
:10F200000075B0FFE5BF5480701C90F1FB74009353
:10F21000C39407500BC374009344B8F59F02F25592
:10F22000759FBC02F255C390F1FD74009394FF707A
:10F230000EC390F1FC74009394FF700302010090E0
:10F24000F1FD740093F5F090F1FC740093F5828564
:10F25000F0837400737581C075C80075CD0075CCDE
:10F260000075CB0075CA0020B0FD30B0FD75C83404
:10F2700020B0FD75C80030B0FD85CD7585CC74E536
:10F280007423235403F574E575232354FC2574F586
:10F2900074E57523235403F575C374009574F574F0
:10F2A00074009575F5758575CD8574CC8575CB85A0
:10F2B00074CA75985A75C834C298D299753479123F
:10F2C000F2D83099FD3098FD02F34D75985A75CB00
:10F2D000FF75CAFA75C834223099FDE534C299F534
:10F2E0009922E542C412F2FEE54212F2FEE543C461
:10F2F00012F2FEE54312F2FE75346851D822540F23
:10F30000C0E0C3940A10D7092441F53451D8D0E0A5
:10F3100022D0E02430F53451D822C0337533FAE5D9
:10F320008954F04401F589756100C28C758CB875FB
:10F330008A02C28DD28C20980C308DFAD533EB75B1
:10F340006101D03322C298859941D03322002098A0
:10F3500005C29902F406C298D299C3E599942A602D
:10F360000302F3F412F6F46035F5F0C3945470140C
:10F3700075343F12F2D875345412F2D8749312F2E5
:10F38000D802F406E5F0C39453C375343F12F2D8A3
:10F3900075345312F2D8749212F2D802F4067880BF
:10F3A00086E0C39446603886E0C3944770028123A8
:10F3B000788086E0C39457602986E0C39452602524
:10F3C00086E0C39445602186E0C39453601D86E0C7
:10F3D000C3944C601986E0C39450601502F3F402A4
:10F3E000F40B02F4DB02F47C02F56502F5B402F6DC
:10F3F000B102F61575343F12F2D875344312F2D8C3
:10F4000075348212F2D8C29802F2C5759F00753425
:10F410004612F2D875345812F2D875349E12F2D8CA
:10F4200002F406759F00088683088682753447516A
:10F43000D875343051D875347751D83099FDC29988
:10F44000C29878027700D8FC758900758C00758A9F
:10F450000075C80075CD0075CC0075CB0075CA006D
:10F4600075F000759800758107E58360028173E58A
:10F4700082600374007302F22602F3F4759F007831
:10F4800081864408864590F1FF740093C3540C9420
:10F490000C700281AB75342112F2D875345212F21D
:10F4A000D87473F53412F2D802F406854483854586
:10F4B00082C3E58394F230D7DCC3740093F54675BC
:10F4C000345212F2D8C374522546F5F085463412F0
:10F4D000F2D885F03412F2D802F406759F007881D4
:10F4E000864408864508864690F1FF7400935403CD
:10F4F000C39403601675345712F2D875345212F261
:10F50000D824A9F53412F2D802F406C3E54494F2E3
:10F5100030D7E2C375F65575F6AA75F65575BF0472
:10F520008544F48545F58546F675F78085448385E1
:10F530004582740093C39546701575345712F2D8FE
:10F5400075343012F2D875348712F2D802F4067589
:10F55000345712F2D875342112F2D82478F53412C7
:10F56000F2D802F406759F0075F65575F6AA75F681
:10F570005575BF0475F783900000C374009394FF22
:10F58000701DA3C3E58394F070F075344512F2D872
:10F5900075343012F2D875347512F2D802F406754B
:10F5A000344512F2D875342112F2D875344512F26E
:10F5B000D802F406759F0078818644C3E54494F12F
:10F5C00030D70EC390F1FF740093C3543094306071
:10F5D0001675345312F2D875345212F2D874A5F558
:10F5E0003412F2D802F40675F65575F6AA75F6557A
:0FF5F00075BF048544F475F50075F782753453C3
:10F5FF0012F2D875343012F2D87483F53412F2D86F
:10F60F0002F40602F69C759F007980788186440883
:10F61F00864508866A90F1FF740093C354039403E0
:10F62F00601875345012F2D875345212F2D87450E3
:10F63F002452F53412F2D802F40608C3E54494F2CA
:10F64F0030D7DFC375F65575F6AA75F65575BF0435
:10F65F008544F48545F586468546F675F7808544DD
:10F66F0083854582740093C395467021080545E54F
:10F67F004570020544D56AC375345012F2D87534FB
:10F68F003012F2D875348012F2D802F40675345065
:10F69F0012F2D875342112F2D875347112F2D802E1
:10F6AF00F406759F0075F65575F6AA75F65575BF74
:10F6BF00040000000075F78175344C12F2D87534D0
:10F6CF003012F2D875347C12F2D802F40675344C2D
:10F6DF0012F2D875343012F2D875349D12F2D80266
:10F6EF00F406745422756100711A8561E070F38518
:10F6FF00413785413B753A2A7880E53A2541F53AFD
:10F70F00711A8561E070DBA64108C3E894CF60D21F
:10F71F00C3D537E6883C18883D18883E18883FA81F
:0DF72F003DE6C3953A600374532274002236
:10FA0000C0E0C083C082C0D0C0BF90F1FF7400933B
:10FA100054039403600D7CF0D0BFD0D0D082D0834B
:10FA2000D0E022C3EF94F010D70D7C0FD0BFD0D020
:10FA3000D082D083D0E022EFC3944030D70EC37C75
:10FA40000FD0BFD0D0D082D083D0E02275F65575CC
:10FA5000F6AA75F65575BF048FF48EF58DF675F719
:10FA6000808F838E82740093FDC39D700D7C00D0C7
:10FA7000BFD0D0D082D083D0E0227CFFD0BFD0D006
:07FA8000D082D083D0E02208
:10FB0000C0E0C083C082C0D0C020C0BF90F1FF74ED
:10FB10000093543003030303C2D79403600F7CF0B7
:10FB2000D0BFD020D0D0D082D083D0E022EFC394F9
:10FB3000EF10D70F7C0FD0BFD020D0D0D082D08391
:10FB4000D0E022EFC3944030D710C37C0FD0BFD099
:10FB500020D0D0D082D083D0E02275F65575F6AA99
:10FB600075F65575BF048FF475F50075F7828F2013
:10FB7000052005208F83758200740093C394FF7065
:10FB800017A3C3E583952070F07C00D0BFD020D0B0
:10FB9000D0D082D083D0E0227CFFD0BFD020D0D084
:07FBA000D082D083D0E022E7
:00000001FF
